:100000000C308A002E2C000045346C3465346B347F
:10001000743472346F346E34693463346B34FD3449
:1000200020346B346F346D34703461347334303455
:100030000D340A340034311CB015E2060A00311CBC
:10004000B016E2060A00331BB016E2060A00453479
:100050006C3465346B34743472346F346E34693498
:1000600063346B34FD3420346B346F346D3470344E
:10007000613473340D340A34003445346C346534DF
:100080006B34743472346F346E34693463346B346B
:10009000FD3420346B346F346D3470346134733418
:1000A00020340D340A340034D3346D38EC32202A35
:1000B000E832F236EF36653AE8327210A51830179A
:1000C0003233A0060A00D3346D38EC32202AE832ED
:1000D000F236EF36653AE832723CA0124C32A00696
:1000E0000A00D3346D38EC32202AE832F236EF368B
:1000F000653AE832F23CA0124C32A0060A00D33432
:100100006D38EC32202AE832F236EF36653AE832C2
:10011000723DA0124C32A0060A008316861183128B
:1001200086110830F80094280000F817A528F81365
:10013000C00C03188615031C86117817A5287813A0
:10014000F80B9828A328000086153F308400840B04
:10015000A7280000F81B9728781B9F280800831603
:1001600003178C170C140000000083128C0803196D
:10017000D2280D080313BD0003170F080313BE0098
:1001800003170C080313C0008D203D0803178D00D2
:1001900003133E0803178F008D0A03198F0A0313F8
:1001A000AF280317031308000830F800000086107A
:1001B0008316861000008312C20D0610031CE3286C
:1001C0008316061483120318E82883160610831278
:1001D000831686148312861CEB28F80BD6280000A1
:1001E0008610831686100000061400000000861496
:1001F0008312861CF928F80100000618781486106E
:1002000083168610831206108316061083120800C8
:10021000303084008313000803191B290230F800D2
:10022000F701F70B1129F80B10299730F700F70B9E
:100230001729800B0E290800831606140000861467
:100240000000831206108316061000008312861029
:10025000831686103C308312C200D420C201D42001
:100260007030C200D420831606100000861483125A
:10027000861C382900003C29000083160614000063
:1002800006308312B000082183160614000086147D
:1002900000008312061083160610000083128610D9
:1002A000831686103C308312C200D4200130C20075
:1002B000D420E030C200D42083160610000086143B
:1002C0008312861C6129000065290000831606142C
:1002D000000006308312B0000821831606140000C7
:1002E0008614000083120610831606100000831285
:1002F0008610831686103C308312C200D420023050
:10030000C200D420C201D420831606100000861437
:100310008312861C892900008D290000831606148B
:10032000000006308312B00008218A150A129E2CA4
:10033000831606140000861400008312061083162C
:100340000610000083128610831686103C3083123C
:10035000C200D4204108C200D42083160610000039
:1003600086148312861CB2290000B6290000831669
:100370000614000006140000861400008312061004
:1003800083160610000083128610831686103D30F7
:100390008312C200D420F7010830C3007708C400DC
:1003A00083160614000086148312861CD5290618AD
:1003B0000314061C0310F80D000083168610831228
:1003C0008610C30BD0298316061400008312061072
:1003D00044080319EE2983160610831200008316C1
:1003E00086148312861CF22900008610831686105C
:1003F0000000831206108316061078088312C100CD
:100400004108F8000800C6014108C500C600C50142
:1004100042084507F8004608FA000318FA0A780867
:10042000C3007A08C4004308F8004408F900080033
:100430008E30F7004208F8004108F900FA01C21FA7
:10044000262AF809F909F90A0319F80AF808031D18
:10045000332A7908F800F9010830F702F808031D7B
:10046000332AF7013C2A0310F81B3A2AF90DF80D3C
:10047000F703332AC21FF813080052080319022B8E
:10048000DE0056080319022BDE02031C4C2A7F30C3
:10049000DE070318022B522A8130DE02031C022BD6
:1004A0000319022B5E08F700F801F901FA01DD01DA
:1004B0005308DC00DC175408DB005508DA0019305B
:1004C000DE005908DA020318752A0130DB0203182E
:1004D000752ADC020318752ADD020318752ADD0A65
:1004E000DC0ADB0A5908DA07A72A5808DB020318D6
:1004F000902A0130DC020318902ADD020318902AAA
:10050000DD0ADC0A5808DB075908DA07031CA72AAA
:10051000DB0A031DA72ADC0A031DA72ADD0AA72A76
:1005200057088038DC020318A62A0130DD020318C0
:10053000A62ADD0A57088038DC075808DB07031CA9
:10054000842ADC0A031D842ADD0A842A7A14DE0B3D
:10055000AA2AB52A0310DA0DDB0DDC0DDD0D031020
:10056000FA0DF90DF80DDF0D612A5F1CBD2A03108D
:10057000F80CF90CFA0CDF0CC02AF7030319022B54
:10058000DF1BE92A0310DA0DDB0DDC0DDD0D590848
:10059000DA020318D52A0130DB020318D52ADC025F
:1005A0000318D52ADD02031CF82A5808DB020318B9
:1005B000E02A0130DC020318E02ADD02031CF82ADD
:1005C00057088038DC020318E92A0130DD02031CD9
:1005D000F82AFA0A031DF82AF90A031DF82AF80A6C
:1005E000031DF82AF70A0319022BF80CF90CFA0C70
:1005F0005308DE005708DE06DE1F002BF817062B17
:10060000F813062BF701F801F901FA0108004F0869
:10061000D6005308D606D61F122B03110310CF1B8A
:100620000314452B4F08D6005208D7004E08D702B6
:100630000319202BD61F452B0308013A8300452BB5
:100640005308D7004F08D70203192C2BD61F452B70
:100650000308013A8300452B5408D7005008D702FD
:100660000319382BD61F452B0308013A8300452B6D
:100670005508D7005108D7020319442BD61F452B24
:100680000308013A8300452B0310080052080319A0
:10069000B62BDA0056080319B62BDA070318572BC6
:1006A0007F30DA02031CB62B0319B62B5B2B81308B
:1006B000DA070318B62B5A08F700F801F901FA0116
:1006C0005308DE00DE175408DD005508DC00183042
:1006D000DA00DB015C1C842B5908FA07031C762B1B
:1006E000F90A031D762BF80A0319DB175808F907D6
:1006F000031C7D2BF80A0319DB175708D400D41705
:100700005408F8070318DB17DB0DF80CF90CFA0C8A
:10071000DE0CDD0CDC0C0310DA0B692B0130F70763
:100720000318B62BF81B9B2BDE0DFA0DF90DF80DF7
:10073000F7030319B62BDE1FAC2BFA0A031DAC2BF3
:10074000F90A031DAC2BF80A031DAC2BF80CF90CAD
:10075000FA0CF70A0319B62B5308DB005708DB061F
:10076000DB1FB42BF817BA2BF813BA2BF701F801DB
:10077000F901FA01080080308318D706DC01DD0199
:100780005308DB005708DB0652080319AB2CDA00CC
:10079000F70056080319B42CDA020319502C031C75
:1007A0000E2C5708E000E0175808DF005908DE005B
:1007B000DD010310E00CDF0CDE0CDD0CDA0BD82BB6
:1007C000DB1FE52B5C14C82C5C105A105C165530EE
:1007D00084008313DD2C5C12DB1BF82B5A1C032CCA
:1007E000E00CDF0CDE0CDD0CF70A0319C32C032C24
:1007F000E01B062C0310DD0DDE0DDF0DE00DF70311
:100800000319C32CF82B5C17702C5C135308DB0006
:10081000DB1F0C2CE017BC2CE013BC2C5608DA00B4
:10082000F7005208DA025308E000E0175408DF002E
:100830005508DE00DD010310E00CDF0CDE0CDD0CE2
:10084000DA0B1A2CDB1F272CDC14C82CDC105A10F6
:10085000DC16593084008313DD2CDC12DB1B3A2CB0
:100860005A1C452CE00CDF0CDE0CDD0CF70A0319DA
:10087000C32C452CE01B482C0310DD0DDE0DDF0DD5
:10088000E00DF7030319C32C3A2CDC17702CDC1392
:100890005708DB00DB1F4E2CE017BC2CE013BC2CF0
:1008A0005708E000E0175808DF005908DE00DB1F9A
:1008B0005D2CE0135C15C82C5C11DD015A1055301D
:1008C00084008313DD2CDB1B862C5308DB005A1CB1
:1008D000702CE00CDF0CDE0CDD0CF70A0319C32CC6
:1008E000DD1F812CDE0A031D812CDF0A031D812CF4
:1008F000E00A031D812CE00CDF0CDE0CF70A031963
:10090000C32C5C1B052CDC1B472CA52C8030E0067F
:10091000E01F8E2CC82C5708DB009B2C5308DB00F3
:10092000E008031D9B2CDF08031D9B2CDE08031D24
:100930009B2CF701BC2CE01BA52C0310DD0DDE0D5C
:10094000DF0DE00DF70B9B2CC32CDB1FA92CE01750
:10095000BC2CE013BC2C5608F7005708E0005808E0
:10096000DF005908DE00BC2C5208F7005308E000F5
:100970005408DF005508DE006008F8005F08F90041
:100980005E08FA00FB2CF701F801F901FA01FB2CD3
:10099000DD01DE09DF09E009DD09DD0A031DD62CD2
:1009A000DE0A031DD62CDF0A0319E00A5C18E42BCB
:1009B000DC18262C5C195C2C8B2C0008DE07031C31
:1009C000E72CDF0A031DE72CE00A03195A148403FD
:1009D0000008DF07031CEF2CE00A03195A148403F4
:1009E0000008801F803AE00703185A145C1AEB2BAA
:1009F000DC1A2D2C632C0800831603178C170C149B
:100A00000000000083120C087F390319402D0313E6
:100A1000BD0003170D080313BE0003170F080313CF
:100A2000BF003D08C0008D203E0803178D00031352
:100A30003F0803178F0083168C170C14000000006A
:100A400083120C0D0E0D7F390319402D0313BD00C9
:100A500003170D080313BE0003170F080313BF008D
:100A60003D08C0008D203E0803178D0003133F088A
:100A700003178F008D0A03198F0A0313FC2C031729
:100A800003130800831603178C170C1400000000D2
:100A90000318712D83120C087F390313B00003175C
:100AA0000D080313B10003170F080313B200300839
:100AB000C0008D20310803178D000313320803177F
:100AC0008F0083168C170C14000000008312031390
:100AD000AF0B6B2D6E2D83160317712D902D831682
:100AE000031783120C0D0E0D7F390313B00003178B
:100AF0000D080313B10003170F080313B2003008E9
:100B0000C0008D20310803178D000313320803172E
:100B10008F008D0A03198F0A03100313AF0B422DA8
:100B20000800F701F801F901FA01C401C501C60185
:100B3000C70143084204410440040319CF2D20306B
:100B4000C8000310BC0DBD0DBE0DBF0DC40DC50DFD
:100B5000C60DC70D43084702031DB82D42084602C3
:100B6000031DB82D41084502031DB82D400844025D
:100B7000031CC92D4008C4024108031C410FC502D3
:100B80004208031C420FC6024308031C430FC7025E
:100B90000314F70DF80DF90DFA0DC80BA12D443013
:100BA0008400831308000408B4003308B600031956
:100BB000F22D3208D5003108D4003008D3002F08B8
:100BC000D200D901D8012030D7008230D600462388
:100BD0007A08B2007908B1007808B0007708AF0051
:100BE000B60BD92D3208BF003108BE003008BD0059
:100BF0002F08BC003C08B63CBC00FA013D08C00010
:100C0000BD170310BD0CBE0CBF0CFA0CF90CF80C90
:100C1000F70CBC0B012EC01F182EF709F809F909B3
:100C2000FA09F70A0319F80A0319F90A0319FA0A63
:100C30007A08B2007908B1007808B0007708AF00F0
:100C4000B21F2F2EB403B416AF09B009B109B2090F
:100C5000AF0A0319B00A0319B10A0319B20A3B30EB
:100C6000BB009A30BA00CA30B900B8010A30B600E9
:100C700033080319B40A3208BF003108BE00300837
:100C8000BD002F08BC003B08C3003A08C200390869
:100C9000C1003808C00091250008AF00840A000890
:100CA000B000840A0008B100840A0008B200FD30D8
:100CB0008407F708031D6F2E330A360203196F2EBF
:100CC00034080319712E0F3936020319692E0318DF
:100CD000A12EB41BA12E341B712E20309D2E20304E
:100CE000B405B41E7F2EB4123308031DB403770875
:100CF000B4002D30C0008D203408F700B401330853
:100D00003602031D8D2E7708B4002E30C0008D20D2
:100D10003408F7002030B40500303030B41E9D2E6A
:100D2000B4123308031DB4037708B4002D30C0009B
:100D30008D203408F700B4013030F7077708C00081
:100D40008D203B08BF003A08BE003908BD003808B6
:100D5000BC00C301C201C1010A30C00091257A085C
:100D6000BB007908BA007808B9007708B800B60B5C
:100D70003B2E8A150A12CB2CB7010408B600371097
:100D8000831B3714B01FCC2EB617361EB60AAF0918
:100D9000B009AF0A0319B00A300EF038B200B2073A
:100DA000E23EB300323EB50030080F39B307B30757
:100DB000B507E93EB400B407B4072F0E0F39B407E6
:100DC000B507B40DB50DB509B50D2F080F39B50729
:100DD000B20D0730B1000A30B507B403031CEC2E86
:100DE000B407B303031CF02EB307B203031CF42EA5
:100DF000B207B103031CF82E31308400831307308F
:100E00003605361384033605031D0D2F361A840A62
:100E1000361A0D2F2030F7002A2F840735300402B0
:100E2000031936170008F700031D1E2F361B1E2F4F
:100E3000361A382FB6191E2F2030292FB61F262F0D
:100E40002D30F70084033613B6132A2FB615361249
:100E50003030F707B0010408AF003010831B3014A6
:100E60007708C0008D202F08840083133018831763
:080E7000840A361F0E2F080052
:101000000330C1008A1198218A157808BD00043088
:10101000C1008A1198218A157808BE003D08C100D8
:101020003E08C2008A1103228A157908C000780898
:10103000BF003F08F8004008F9007908B0007808C0
:10104000AF000730C1008A1198218A157808BD00C9
:101050000830C1008A1198218A157808BE003D0821
:10106000C1003E08C2008A1103228A157908C00017
:101070007808BF003F08F8004008F9007908B2007E
:101080007808B1000530C1008A1198218A157808C6
:10109000BD000630C1008A1198218A157808BE006B
:1010A0003D08C1003E08C2008A1103228A15790852
:1010B000C0007808BF003F08F8004008F900790830
:1010C000B4007808B3003208C2003108C1008A11A8
:1010D00018228A157708BD007808BE007908BF007D
:1010E0007A08C0003008C2002F08C1008A111822F7
:1010F0008A154008D5003F08D4003E08D3003D08BB
:10110000D2007A08D9007908D8007808D700770883
:10111000D6008A113D228A157A08B8007908B700EE
:101120007808B6007708B5003808C0003708BF0057
:101130003608BE003508BD004D10CD104008C40073
:101140003F08C3003E08C2003D08C1004008D1006E
:101150003F08D0003E08CF003D08CE00D501D401A5
:10116000D301D2018A1107238A15031CBB284D1411
:101170004208803AC200D101D001CF017F30CE00B9
:101180004408D5004308D4004208D3004108D200E7
:101190008A1107238A15031CE628D501D401D3013F
:1011A0007F30D2004408D9004308D8004208D70055
:1011B0004108D6008A113D228A157A08C4007908B0
:1011C000C3007808C2007708C100CD140A30D500EA
:1011D0008930D4003430D3007C30D2004408D900A8
:1011E0004308D8004208D7004108D6008A11462398
:1011F0008A157708CE007808CF007908D0007A08E1
:10120000D100D5007908D4007808D3007708D2003F
:101210004408D9004308D8004208D7004108D60046
:101220008A1146238A157708CE007808CF007908FE
:10123000D0007A08D10083107A08D5007908D4004C
:101240007808D3007708D2007C30D9007930D800F4
:101250003530D7008130D6008A11BB238A157A0831
:10126000C8007908C7007808C6007708C500480894
:10127000D5004708D4004608D3004508D2004408EA
:10128000D9004308D8004208D7004108D6008A1187
:1012900046238A157708CE007808CF007908D00059
:1012A0007A08D100D5007908D4007808D3007708EF
:1012B000D2004408D9004308D8004208D7004108AA
:1012C000D6008A1146238A157708CE007808CF0009
:1012D0007908D0007A08D10083107A08D5007908FF
:1012E000D4007808D3007708D2003F30D90002300C
:1012F000D8003330D7008330D6008A11BB238A153B
:101300007A08C8007908C7007808C6007708C500C1
:101310004808D5004708D4004608D3004508D20045
:101320004408D9004308D8004208D7004108D60035
:101330008A1146238A157708CE007808CF007908ED
:10134000D0007A08D100D5007908D4007808D300FD
:101350007708D2004408D9004308D8004208D700D3
:101360004108D6008A1146238A157708CE007808EE
:10137000CF007908D0007A08D10083107A08D50010
:101380007908D4007808D3007708D2003330D90028
:101390008C30D8001E30D7008330D6008A11BB2392
:1013A0008A157A08C8007908C7007808C600770847
:1013B000C500D501D401D3017F30D2004408D90043
:1013C0004308D8004208D7004108D6008A114623B6
:1013D0008A157708CE007808CF007908D0007A08FF
:1013E000D100D5007908D4007808D3007708D2005E
:1013F0004408D9004308D8004208D7004108D60065
:101400008A1146238A157708CE007808CF0079081C
:10141000D0007A08D10083107A08D5007908D4006A
:101420007808D3007708D2001B30D900E430D80008
:101430003530D7008230D6008A11BB238A157A084E
:10144000CC007908CB007808CA007708C9004C089E
:10145000D5004B08D4004A08D3004908D2004408FC
:10146000D9004308D8004208D7004108D6008A11A5
:1014700046238A157708CE007808CF007908D00077
:101480007A08D100D5007908D4007808D30077080D
:10149000D2004408D9004308D8004208D7004108C8
:1014A000D6008A1146238A157708CE007808CF0027
:1014B0007908D0007A08D10083107A08D50079081D
:1014C000D4007808D3007708D200A430D900DB30EC
:1014D000D8006730D7008330D6008A11BB238A1525
:1014E0007A08CC007908CB007808CA007708C900D0
:1014F0004C08D5004B08D4004A08D3004908D20054
:101500004408D9004308D8004208D7004108D60053
:101510008A1146238A157708CE007808CF0079080B
:10152000D0007A08D100D5007908D4007808D3001B
:101530007708D2004408D9004308D8004208D700F1
:101540004108D6008A1146238A157708CE0078080C
:10155000CF007908D0007A08D10083107A08D5002E
:101560007908D4007808D3007708D2003330D90046
:101570008C30D8001E30D7008330D6008A11BB23B0
:101580008A157A08CC007908CB007808CA00770859
:10159000C9004408D5004308D4004208D3004108DC
:1015A000D2004808D9004708D8004608D7004508A7
:1015B000D6008A1146238A157708CE007808CF0016
:1015C0007908D0007A08D100D5007908D4007808CD
:1015D000D3007708D2004C08D9004B08D8004A083D
:1015E000D7004908D6008A113D228A157A08C8001A
:1015F0007908C7007808C6007708C500CD1C1C2BE9
:101600008314DB30D5000F30D4004930D3007F3055
:10161000D2004808D9004708D8004608D700450836
:10162000D6008A11BB238A157A08C8007908C7003A
:101630007808C6007708C5004D1C212B4608803A63
:10164000C6004508F7004608F8004708F9004808B2
:10165000FA007A08BC007908BB007808BA0077085D
:10166000B9003C08D5003B08D4003A08D30039083B
:10167000D200C330D900F530D8004830D7008030D0
:10168000D6008A113D228A157708BD007808BE0071
:101690007908BF007A08C000D5003F08D4003E0892
:1016A000D3003D08D200D901D8013430D7008630AC
:1016B000D6008A1146238A157A08BC007908BB0037
:1016C0007808BA007708B9003908F7003A08F80036
:1016D0003B08F9003C08FA00F8133C08BC003B0842
:1016E000BB007808BA003908B900AF08031D9B2B6E
:1016F000B008031D9B2B043003178D0000308F00B2
:101700008A110313AF208A15B21B942BB208031D54
:101710008D2B3108003C0318942BBC01BB013430E5
:10172000BA008530B9009A2BBC01BB010730BA0062
:101730008730B900232CB01BEE2BB008031DA42B5F
:101740002F08003C0318EE2BB21BCA2B8310D501C7
:10175000D4013430D3008630D2003C08D9003B0895
:10176000D8003A08D7003908D6008A11BB238A1559
:101770007A08BC007908BB007808BA007708B9007D
:101780001B3003178D0000308F008A110313FC24D7
:101790008A15ED2B8314D501D4013430D300863063
:1017A000D2003C08D9003B08D8003A08D7003908D5
:1017B000D6008A11BB238A157A08BC007908BB00C1
:1017C0007808BA007708B9001F3003178D00003081
:1017D0008F008A110313FC248A15232CB21B142CAE
:1017E0008314D501D4013430D3008730D2003C08B3
:1017F000D9003B08D8003A08D7003908D6008A112A
:10180000BB238A157A08BC007908BB007808BA00A7
:101810007708B900233003178D0000308F008A113C
:101820000313FC248A15232C6230C0008A118D20FA
:101830008A150D30C0008A118D208A150A30C0002B
:101840008A118D208A153908F7003A08F8003B08FC
:10185000F9003C08FA008A150A12A02C84018313AF
:101860001F308305713083168F000F088611831295
:101870008615831603170908C039890003131F1240
:101880009F120030031788008312870188018901A5
:10189000FF300313A000831603170908C03989001D
:1018A00003131F129F1200300317880083120313C3
:1018B0001F139F1383169F1383121F149412A012D9
:1018C00020088316870083122016200883168700BD
:1018D0008312A01120088316870001308312940020
:1018E0000030831694000108C7390838810083123C
:1018F00090010030F80092000030831692008312AD
:1019000020152008831687008312970183169B01F8
:101910009C0101309D008312031787018801890112
:1019200027308D0000308F008A110313AF208A15F5
:10193000A801A701A601A5018A111C298A15002862
:101940007A08A4007908A3007808A2007708A1000B
:101950003D3003178D0000308F008A110313AF2034
:101960008A15543003178D0000308F000310143097
:101970000313AF008A1142258A1509308400240818
:10198000B2002308B1002208B0002108AF000230E5
:10199000B3008A11D32D8A152030C0008A118D2002
:1019A0008A150D30C0008A118D208A150A30C000BA
:1019B0008A118D208A15633003178D0000308F0047
:1019C000031015300313AF008A1142258A15103019
:1019D00084002A08B0002908AF008A11BC268A15A5
:1019E0002030C0008A118D208A150D30C0008A1168
:1019F0008D208A150A30C0008A118D208A15713019
:101A000003178D0000308F00031015300313AF0053
:101A10008A1142258A15103084002C08B0002B084A
:101A2000AF008A11BC268A152030C0008A118D2093
:101A30008A150D30C0008A118D208A150A30C00029
:101A40008A118D208A157F3003178D0000308F009A
:101A5000031015300313AF008A1142258A15103088
:101A600084002E08B0002D08AF008A11BC268A150C
:101A70002030C0008A118D208A150D30C0008A11D7
:101A80008D208A150A30C0008A118D208A150830F1
:101A9000AF00FA30B0008A1108218A15AF0B492D2A
:041AA0009F2C630014
:04400E00F52CFF3F4F
:00000001FF
